:103800000C94341C0C944F1C0C944F1C0C944F1CA7
:103810000C944F1C0C944F1C0C944F1C0C944F1C7C
:103820000C944F1C0C944F1C0C944F1C0C944F1C6C
:103830000C944F1C0C944F1C0C944F1C0C944F1C5C
:103840000C944F1C0C944F1C0C944F1C0C944F1C4C
:103850000C944F1C0C944F1C0C944F1C0C944F1C3C
:103860000C944F1C0C944F1C11241FBECFEFD4E0BE
:10387000DEBFCDBF11E0A0E0B1E0EEE4FFE302C0A7
:1038800005900D92A430B107D9F712E0A4E0B1E0A1
:1038900001C01D92A634B107E1F70C94691F0C9486
:1038A000001C0F92AF93BF93CF93DF93EF93FF93DF
:1038B000FC01EA01DB01C895099231961197D9F70D
:1038C000FF91EF91DF91CF91BF91AF910F9008954C
:1038D0000F921F920F93AF93BF93CF93DF93EF930A
:1038E000FF93FC01EA01DB010990199001E043D04C
:1038F00032961297C9F7FC0103E03DD005E03BD0BA
:10390000FF91EF91DF91CF91BF91AF910F911F90F8
:103910000F9008950F931F93EF93FF93FC0103E023
:103920002AD000E810E0E00FF11FE617F707B9F71B
:10393000FF91EF911F910F9108950F930F9222D055
:10394000082E09E018D00F900F9108950F930F9251
:10395000EF93FF9317D0FC0160935700C895802D1B
:10396000FF91EF910F900F9108950F930BD001E10C
:1039700002D00F910895F999FECF00935700E89572
:10398000FFFF00000091570000FDFCCF08958AE082
:103990008093C4008091C10088618093C100089524
:1039A0008091C100877E8093C10008958093C600F6
:1039B0008091C00086FFFCCF8091C000806480931E
:1039C000C00008958091C600992708958091C00095
:1039D0009927807890700895EF92FF920F931F932C
:1039E000CF93DF937B01C0E0D0E0C617D70770F418
:1039F0008C010E94E61C8823E1F30E94E21CF8017E
:103A000081938F012196CE15DF0598F381E090E038
:103A1000DF91CF911F910F91FF90EF900895EF925A
:103A2000FF920F931F93CF93DF937C018B01C0E034
:103A3000D0E0C017D10738F4F70181917F010E94CF
:103A4000D61C2196F6CF81E090E0DF91CF911F91B7
:103A50000F91FF90EF900895EF92FF920F931F93B5
:103A6000CF93DF937C0100E010E00817190788F47A
:103A7000C0E0D0E000000E94E61C882351F42196AB
:103A800089E0C43CD807B0F30F5F1F4F0E151F0528
:103A900078F3DF91CF911F910F91FF90EF900895F0
:103AA0000E94D01C0E9400000895DF92EF92FF92C6
:103AB0000F931F93CF93DF93CDB7DEB72197DEBF70
:103AC000CDBF8C017B011982D98061E070E0CE010D
:103AD000860F971F0E94EC1C89818B31B1F761E042
:103AE00070E0C8010E94EC1C61E070E0CE01860F1E
:103AF000971F0E94EC1C89819927182F002761E0ED
:103B000070E0CE01860F971F0E94EC1C8981080F80
:103B1000111D61E070E0CE01860F971F0E94EC1C22
:103B200089818E30B9F4C8010196BC01C7010E9499
:103B3000EC1C98018FEF0F3F180779F0F701819186
:103B40007F01D82621503040FFEF2F3F3F07B1F7CC
:103B5000DD2019F080E090E001C0C8012196DEBFB1
:103B6000CDBFDF91CF911F910F91FF90EF90DF902C
:103B70000895CF92DF92FF920F931F93CF93DF931D
:103B8000182FEB016A018BE10E94D61C4BE1F42E49
:103B9000812F0E94D61CF1260D2F1127802F0E9405
:103BA000D61CF0268C2F0E94D61CFC268EE00E948C
:103BB000D61C8EE0F82621978FEFCF3FD80759F01B
:103BC000F60181916F01F8260E94D61C2197FFEF24
:103BD000CF3FDF07A9F78F2D0E94D61CDF91CF9131
:103BE0001F910F91FF90DF90CF9008959927813911
:103BF000910559F08239910524F48039910529F015
:103C000008C08239910519F004C082E003C087E042
:103C100001C080EC99270895BF92CF92DF92EF9276
:103C2000FF920F931F93CF93DF93B82E8B01FB016D
:103C30008081C82FDD27C231D10509F46DC0C331A1
:103C4000D105DCF4C330D10509F44DC0C430D10531
:103C500044F4C130D10579F1C230D10509F44AC02C
:103C600004C1C630D10509F44AC0C630D1050CF4F0
:103C7000FCC060970CF4F9C055C0C531D10509F4FA
:103C8000C8C0C631D10544F4C331D10509F472C0AE
:103C9000649709F44AC0E9C0CA31D10509F4D7C014
:103CA000CB31D10524F4669709F49AC0DEC06B9736
:103CB00009F4C4C0DAC0FB01118288E0828381E488
:103CC000838386E5848382E5858389E4868383E52F
:103CD000878380E580878FE5818782E38287AB01D8
:103CE0006BE070E0C8C0FB0181810E94F61DF80105
:103CF000828301C0FB011182A801BE01BCC0FB018F
:103D000083819927982F88272481820F911D909372
:103D100045028093440207C060E070E480E090E0D8
:103D20000E948A1CF8011182A3C0FB01818199279E
:103D3000D82FCC2782819927C82BD92B1182CB0170
:103D400002962091440230914502AC01BE01C901A6
:103D5000880F991F0E94511CF801EC0FFD1F128261
:103D60009E01369527958091440290914502820FDD
:103D7000931F49C0FB0181819927D82FCC278281CD
:103D80009927C82BD92BCC24DD24CC16DD06D8F4FA
:103D9000FAE0EF2EF12CE60EF71E8091440290918E
:103DA0004502880F991FA70160E870E08C0D9D1DEA
:103DB0000E94681C80E890E0C80ED91EE80EF91E2B
:103DC000CC16DD0650F30E94B51CF8011182D69581
:103DD000C79580914402909145028C0F9D1F29C088
:103DE000FB0181819927D82FCC2782819927C82B65
:103DF000D92B1182EC0FFD1F128280914402909109
:103E000045028C0F9D1F9093450280934402239698
:103E100073CFFB0181819927382F2227828199272F
:103E2000282B392B11828091440290914502820FF8
:103E3000931F90934502809344021AC0FB011182A4
:103E40008481E82FFF27E050FF4F808107C0FB01EE
:103E5000118269E081E090E00E94A61CF801828353
:103E60001382A80164E070E006C089ECF801818348
:103E7000A80162E070E08B2D0E94B91DDF91CF9107
:103E80001F910F91FF90EF90DF90CF90BF9008951A
:103E9000CF93DF93CDB7DEB72197DEBFCDBF69E00B
:103EA00081E090E00E94A61C992784FF09C08F7EC4
:103EB0000E949D1C05C064E071E089810E940C1E77
:103EC00064E071E0CE0101960E94551D892B99F3A3
:103ED000F7CFCFEFD4E0DEBFCDBFCEE1F894AEEFA9
:103EE000B1E00E949E1F802D843B79F4AFEFB1E0DA
:103EF0000E949E1F802D833C41F4ADEFB1E00E94F3
:103F00009E1F802D9927809366000E94C71C0E94E7
:103F1000E21C84E690E00E942C1D0E94E61C88238F
:103F200019F00E94481F04C0C150C5B9CC2389F7BD
:103F30000E94501D80E090E00C94A61FF999FECFDE
:0E3F4000B2BDA1BDF89A119600B40895FFCF4E
:043F4E001E940600B7
:0400000300003800C1
:00000001FF
